:100000006DC0DFC186C085C084C083C082C081C08E
:1000100080C07FC07EC07DC07CC07BC07AC079C0FC
:1000200078C077C076C00403090418037200610029
:10003000700068006E00650074002E006E006500A0
:10004000740018035300650067006100200053002E
:1000500061007400750072006E000A033100300008
:100060003000300005010905A10185010901A10049
:100070000930093109360937150026FF0075089542
:10008000048102C005091901291015002501750117
:1000900095108102C005010902A10185020901A193
:1000A0000005091901290415002501950475018130
:1000B00002950175048103C00501093009311581DC
:1000C000257F750895028106C0120101010000001C
:1000D0000881177E050101010203010011241FBEE2
:1000E000CFE5D4E0DEBFCDBF10E0A0E6B0E0E2E7B0
:1000F000F0E102C005900D92A63BB107D9F711E0DF
:10010000A6EBB0E001C01D92AB32B107E1F71AD304
:10011000AEC776CF85B7836085BF8BB780648BBF52
:1001200083EC8093010108950F931F93CF93DF9386
:100130009091110119160CF0A8C020910E01809128
:100140000D018D3209F097C08AE5809361009B30E4
:1001500009F091C0CCE0D0E0C21BD109CB5EDE4FEC
:100160008881807609F079C01092FF008981882308
:1001700059F4109200018FEF90E09093100180935A
:100180000F0130E822E070C0853021F48A8180932D
:10019000120161C0863009F043C08B818130D9F1F2
:1001A000823019F4CE0170D25AC0833039F58A8179
:1001B000882349F486E290E09093100180930F0128
:1001C00030EC24E051C0813019F48AE290E004C0A0
:1001D000823049F482E490E09093100180930F0103
:1001E00030EC28E141C08330E9F58AE590E0909356
:1001F000100180930F0130EC2CE036C0813249F4BD
:1002000089EC90E09093100180930F0130EC29E08D
:100210002BC0823239F5CE0137D2282F30EC24C0E2
:10022000883019F484E191E00AC0893021F48A8190
:100230008093140110C08A3049F48FEF90E09093BE
:10024000100180930F0130E821E00EC08B3019F4CB
:1002500083EC8093010130E806C0CE0143D2282F01
:1002600030E802C030EC20E08F81882339F48E81A1
:10027000821728F003C030E880E001C0822F30935D
:10028000B60080936000109211018091610084FF9C
:1002900049C0809160008F3F09F444C0182F893015
:1002A00008F018E0811B809360008091B60080FD0B
:1002B00002C00BE401C003EC8F5F8093B600209175
:1002C0000F013091100186FD05C0D901912FE7EF94
:1002D000F0E011C0A7EFB0E080E090E006C0F901C7
:1002E000E80FF91FE491ED9301961817C1F705C0C7
:1002F0008D91819391509923D9F7F901E10FF11D67
:10030000F0931001E0930F0187EF90E0612F55D03B
:10031000183019F08FEF809360000093F6001C5F97
:10032000109361009AE080B3857031F49150D9F751
:100330001092120110920C01DF91CF911F910F9139
:1003400008951F93DC01162F8091620084FF0AC07C
:100350008091010198E8892780930101912FE2E0C3
:10036000F1E007C08AE580936200F8CF8D91819318
:1003700091509923D9F782E091E0612F1ED01C5F44
:10038000109362001F910895A82FB92F8FEF9FEF50
:1003900041E050EA615070F02D9138E0722F7827DB
:1003A00096958795269570FF02C0842795273A95E4
:1003B000A9F7F0CF809590950895E6DF8D939D93F2
:1003C0000895CF93CFB7CF93809BFECF809B09C07A
:1003D000809B07C0809B05C0809B03C0809B01C0A1
:1003E0009EC0DF93C0910E01DD27CB5EDE4F809B68
:1003F00002C0DF91EBCF2F930F931F9300B32FEF2A
:1004000000FB20F94F933F9310B34FEF012700FB00
:1004100021F93BE031C04E7F012F10B3216028C08D
:10042000102F4D7F2260000000B329C04B7F246055
:10043000012F000010B32BC010B3477F28602AC0E3
:100440004F7E00B320612CC04F7D10B320622FC0BF
:100450004F7B00B3206432C0422700B349934FEF73
:100460000000102710FB20F910B31570A9F1297FA7
:1004700091F2012700FB21F900B3237F89F231506B
:10048000F0F1102710FB22F910B3277E79F2012733
:1004900000FB23F92F7C81F200B3102710FB24F915
:1004A0002F7971F200C010B3012700FB25F92F73DB
:1004B00059F200C000B3102710FB26F9223040F299
:1004C00000C010B3012700FB27F9243028F64F772E
:1004D000206810B30000F9CF3B503195333010E461
:1004E0001ABFB8F0C31BD0400881033C41F10B3464
:1004F00031F11981412F1F7720910C01121731F42E
:10050000093691F10D3279F0013E69F022272093EE
:1005100013013F914F911F910F912F91DF91CF9137
:10052000CFBFCF911895009313013F914F911F9129
:100530000F912F91DF91CAB7C6FD46CFF0CF009142
:100540001301002331F3109111011123A1F534306F
:10055000A2F13093110100930D0110910E013BE0C7
:10056000311B30930E0129C00091110101301CF59F
:100570000AE547FD09C03091610034FD20C00093B9
:100580006100C6EFD0E01FC03091620034FD17C09B
:1005900000936200C1E0D1E016C0052710E002BB65
:1005A0001FC0052722C0052727C005272CC0052707
:1005B00010E002BB33C04AE503C042ED01C0432F47
:1005C000C4E1D0E032E011B31560909A02B311BBE0
:1005D0005F9355E020E820FF052702BB279517957C
:1005E0001C3FD8F620FF0527279502BB17951C3F17
:1005F000C0F620FF05272795179502BB1C3F98F6EC
:1006000020FF0527279517951C3F02BB70F600C0F9
:10061000499120FF052702BB279517951C3F38F607
:1006200020FF0527279502BB17951C3F38F520FFB3
:1006300005272795179502BB1C3F10F520FF0527BE
:10064000279517951C3F02BBE8F4242F3A9519F61D
:100650000A7F5F9102BB00C010911201C651D040C9
:1006600011F010930C0110E41ABF016011B31A7F4E
:10067000402F4A7F02BB11BB42BB4BCF0527D3CFD4
:100680000527D8CF0527DDCFFC018081807641F595
:100690008181863029F583818230D1F0823269F000
:1006A0008130F1F48091BB009091BC0090931001D7
:1006B00080930F018091BD0008958091B8009091C2
:1006C000B9009093100180930F018091BA000895B2
:1006D00083E690E09093100180930F0182E20895E9
:1006E00080E00895DC0120EC30E03093100120938D
:1006F0000F018C918076803219F511968C911197AB
:10070000813061F4E091BE00F091BF000088F18972
:10071000E02DC90112966C9109950895823041F43B
:1007200080ED90E09093100180930F0181E0089597
:100730008A3031F413968C918093D00080E0089534
:1007400080E008958F929F92AF92BF92CF92DF92F6
:10075000EF92FF920F931F93CF93DF9386B3BCD199
:10076000FC019093BF008093BE008481958190939B
:10077000B9008093B80082818093BA00808591850A
:10078000009731F09093BC008093BB00868107C036
:1007900089EC90E09093BC008093BB004FD4809391
:1007A000BD008091BA0080937C0014BA8FEF85BBA6
:1007B00088EF82BB85E081BB11BA83BF8FE085BD26
:1007C00084EC83BDE091BE00F091BF000284F3850C
:1007D000E02D099585B78F7885BF9CDC789400E083
:1007E000FF24F39410E08824839431E0C32ED12CAD
:1007F00020E8922E9CE2A92E91E0B92E02C0FF249F
:100800001E2DA89591DCFF2041F0E091BE00F091F3
:10081000BF000484F585E02D099508B600FE0DC0E3
:1008200088BEE090D000EE2041F0153010F403E0D7
:1008300005C08BEFE82EE10E01C0E12E08B607FEE1
:1008400033C098BE002399F585B7806885BF889529
:1008500085B78F7785BFC5010197F1F7E091BE009D
:10086000F091BF000484F585E02D0995C0E0D0E04B
:1008700012C00684F785E02D9E012F5F822F099517
:10088000882341F0C6010C2E02C0880F991F0A94DC
:10089000E2F7082B2196E091BE00F091BF00808125
:1008A0009181C817D9072CF3002309F4A8CFC0E021
:1008B000D0E02DC0802F992787FD90950C2E02C087
:1008C000959587950A94E2F780FF20C0CE018F5F4F
:1008D000682F0088F189E02D80EC90E00995182FB1
:1008E00001C022DC8091620084FFFBCF612F77275B
:1008F00067FD709580EC90E024DDC6010C2E02C0EF
:10090000880F991F0A94E2F7809508232196E091B9
:10091000BE00F091BF0080819181C817D90754F2C1
:100920006ECF43B366B350E0CA0184709070959562
:1009300087959A0128703070E3E035952795EA9500
:10094000E1F7822B9A0122703070220F331F822B25
:100950004170507023E0440F551F2A95E1F7842B16
:1009600070E06072707075956795862B08958FB7EB
:10097000F89490E394BB9FEF95BB17BA98BB8FBFD9
:1009800008950F931F93882319F414E604E011C00F
:1009900014E604E005C0802F8A95F1F7115069F044
:1009A000C0DF84FFF8CF0BC0802F8A95F1F711507C
:1009B00021F0B7DF84FDF8CF02C08FEF01C080E0E7
:1009C0001F910F9108950F931F93DF93CF93CDB78E
:1009D000DEB76B970FB6F894DEBF0FBECDBFDE015A
:1009E0001196EDEAF0E089E001900D928150E1F777
:1009F000DE011A96E4EAF0E089E001900D92815060
:100A0000E1F7DE015396EBE9F0E089E001900D9209
:100A10008150E1F78091D700682F70E09091D80065
:100A200080E0682B792B8091D100882391F481E0BC
:100A30008093D10060FF03C082E08093D10061FF0A
:100A400003C083E08093D10062FF03C084E0809301
:100A5000D1008091D100823029F0833049F081307B
:100A600081F503C0DE011A9605C0DE01119602C0B1
:100A7000DE015396AB0140705E7F20E030E001E084
:100A800010E0C801022E02C0880F991F0A94E2F7F5
:100A900086239723892B61F0FD01E20FF31FC80124
:100AA000008002C0880F991F0A94E2F7482B592B47
:100AB0002F5F3F4F2930310521F74093D7005093E6
:100AC000D8006B960FB6F894DEBF0FBECDBFCF91A6
:100AD000DF911F910F91089584E690E090938A0032
:100AE0008093890085E890E008951F93162F115098
:100AF000123010F010E029C0009789F0E12FF0E0EB
:100B0000E956FF4FE081FF27E7FDF09529E0129FAE
:100B1000900111242E523F4FB901AF019FD229E01D
:100B2000129F90011124E12FF0E0E956FF4F108150
:100B3000A9014C515F4FE12FFF27E7FDF0952E52A1
:100B40003F4FCA01B901AF0189D2812F1F9108958A
:100B5000E82F8091990090919A00892B31F01092A2
:100B60009A001092990081E008958E2F8150823072
:100B700010F080E0089569E0869FB0011124E82F0D
:100B8000F0E0E956FF4F4081552747FD5095CB01D6
:100B90008E529F4F6C517F4F54D208959F92AF92C7
:100BA000BF92CF92DF92EF92FF920F931F93DF934A
:100BB000CF93CDB7DEB7A0970FB6F894DEBF0FBEC8
:100BC000CDBFAD9AAC9A30E1F32E8F2D8A95F1F717
:100BD000A8DE982F813109F0F2C089E0EBEDF0E05A
:100BE000DF011D928A95E9F782E08093DB008F2D6B
:100BF0008A95F1F7AD988F2D8A95F1F7FF2400E0E3
:100C000010E02EE0C22ED12CEE2498E0992E5E0149
:100C10000894A11CB11CFF2019F0AC9A81E002C01D
:100C2000AC9880E0AEDE882309F0F6C1892D8A9564
:100C3000F1F777DEF501E00FF11F80830115110553
:100C400041F08A81823129F488E0C82ED12CEE242B
:100C5000E3940F5F1F4F0C151D051CF481E0F8266F
:100C6000DACF91E09093D2008FE78093D300809306
:100C7000D4008093D5008093D6001092D7001092B4
:100C8000D8008C81282F82FD02C09093D70020FDD0
:100C900005C08091D70082608093D70021FD05C0F8
:100CA0008091D70084608093D7008D81982F82FD3A
:100CB00005C08091D70088608093D70091FD05C062
:100CC0008091D70080618093D70090FD05C080910E
:100CD000D70080628093D70023FD05C08091D700A4
:100CE00080648093D7008E8183FD05C08091D700FA
:100CF00080688093D70093FD05C08091D800816003
:100D00008093D8008B81EE20A1F0982F83FD03C043
:100D10008FEF8093D30092FD02C01092D30091FD1B
:100D200003C08FEF8093D40090FD40C01092D40098
:100D30003DC0982F83FD05C08091D80084608093CA
:100D4000D80092FD05C08091D80088608093D800BB
:100D500091FD05C08091D80080618093D80090FDFE
:100D600005C08091D80080628093D8009F819295C1
:100D7000907F88858F70982B9093D300998592955A
:100D8000907F8A858F70982B9093D4009B85929545
:100D9000907F8C858F70982B9093D5009D85929530
:100DA000907F8E858F70982B9093D600AC9A80E1BF
:100DB000982F9A95F1F7AD9A8A95F1F791C08771BE
:100DC000843109F08FC00BED10E089E0F801119239
:100DD0008A95E9F782E08093DB0009501040AD9AD4
:100DE000AC9A8F2D8A95F1F79CDDE82EAD98AC98E2
:100DF0008F2D8A95F1F795DDC82EAD9AAC988F2D81
:100E00008A95F1F78EDDD82EAD98AC9A8F2D8A9504
:100E1000F1F787DD91E09093D2009FE79093D300A4
:100E20009093D400D80113969C93139714969C9397
:100E30001092D7001092D800282F83FD03C08FEFA7
:100E40008093D30022FD02C01092D30021FD03C085
:100E50008FEF8093D40020FD02C01092D4002D2D7E
:100E6000D2FC05C08091D70081608093D70020FD1F
:100E700005C08091D70082608093D70021FD05C016
:100E80008091D70084608093D7009C2DC2FC05C060
:100E90008091D70088608093D70091FD05C0809134
:100EA000D70080618093D70090FD05C08091D70066
:100EB00080628093D70023FD05C08091D7008064B5
:100EC0008093D700E3FC05C08091D70080688093B1
:100ED000D70093FD05C08091D80081608093D80031
:100EE00072DD9AC0E2EDF0E0903109F07CC081E063
:100EF0008093D2008FE78093D3008093D4008093B7
:100F0000D5008093D6001092D7001092D800892F78
:100F10008A95F1F7AD98892F8A95F1F78E010F5FC9
:100F20001F4FFF24B8E0BB2EA9E0CA2ED12CCC0E57
:100F3000DD1EFF2019F0AC9A81E002C0AC9880E081
:100F400020DD882309F068C08B2D8A95F1F7E9DC54
:100F5000F80181938F01EC15FD0519F081E0F82669
:100F6000E8CFAC9A80E1982F9A95F1F7AD9A8A95DF
:100F7000F1F789E0EBEDF0E0DF011D928A95E9F7EA
:100F800082E08093DB008C81982F80FF05C08091E8
:100F9000DC0081608093DC0091FF05C08091DC0063
:100FA00082608093DC0092FF05C08091DC00846049
:100FB0008093DC0093FF05C08091DC008860809303
:100FC000DC002F812295207F88858F70282B9D81C2
:100FD0009295907F8E818F70982B9093DD00219554
:100FE0002093DE0019C081E08093D2008FE78093C8
:100FF000D3008093D4008093D5008093D6001092C4
:10100000D7001092D800399689E0DF011D928A95A9
:10101000E9F782E08093DB00A0960FB6F894DEBF7C
:101020000FBECDBFCF91DF911F910F91FF90EF9039
:10103000DF90CF90BF90AF909F90089582E190E0B5
:101040000895FB01DC0104C08D910190801921F409
:1010500041505040C8F7881B990B0895FB01DC01F3
:1010600002C001900D9241505040D8F70895F89475
:02107000FFCFB0
:10107200FF5A5A09022200010100803209040000CD
:1010820001030000000921010100012200000705FF
:10109200810308000A02006500000000000000B79A
:1010A20004CE05A80575050704010000010203042A
:1010B20005080607010205000304080607010205E8
:0610C2000003040906070B
:00000001FF
